:0200000480007A
:100000006F00C004732F2034930F8000630AFF0336
:10001000930F90006306FF03930FB0006302FF038A
:10002000170F0080130F0FFE63040F0067000F000F
:10003000732F203463540F006F004000136E9E53E3
:10004000171F00002320CFFD6FF09FFF732540F1A5
:100050006310050073251030635805000F00F00F82
:10006000130E100073000000130E00009702000032
:10007000938282F973905230735020307350303035
:1000800073504030970200809382C2F7638C020065
:10009000739052109302B01A739022307323203061
:1000A000E39E62F873500030970200009382420191
:1000B00073901234732540F17300203093000000D8
:1000C00093D10040930E0000130E20006394D12BB7
:1000D000B700008093D11040B70E00C0130E30005F
:1000E000639AD129B700008093D17040B70E00FF0A
:1000F000130E40006390D129B700008093D1E040F7
:10010000B70EFEFF130E50006396D127B700008094
:100110009380100093D1F041930EF0FF130E600016
:10012000639AD125B70000809380F0FF93D10040FF
:10013000B70E0080938EFEFF130E7000639CD123D8
:10014000B70000809380F0FF93D11040B70E0040BD
:10015000938EFEFF130E8000639ED121B7000080B6
:100160009380F0FF93D17040B70E0001938EFEFF95
:10017000130E90006390D121B70000809380F0FFB0
:1001800093D1E040B70E0200938EFEFF130EA00045
:100190006392D11FB70000809380F0FF93D1F041AC
:1001A000930E0000130EB0006396D11DB7808181BD
:1001B0009380101893D10040B78E8181938E1E18C2
:1001C000130EC0006398D11BB780818193801018F3
:1001D00093D11040B7CEC0C0938E0E0C130ED0003A
:1001E000639AD119B78081819380101893D17040A0
:1001F000B70E03FF938E3E30130EE000639CD117C1
:10020000B78081819380101893D1E040B70EFEFF34
:10021000938E6E60130EF000639ED115B7808181BE
:100220009380101893D1F041930EF0FF130E00014C
:100230006392D115B700008093D07040B70E00FFD5
:10024000130E10016398D01313020000B700008052
:1002500093D1704013830100130212009302200017
:10026000E31652FEB70E00FF130E20016314D311E4
:1002700013020000B700008093D1E040130000009B
:10028000138301001302120093022000E31452FEB4
:10029000B70EFEFF130E3001631ED30D13020000D4
:1002A000B70000809380100093D1F041130000004C
:1002B00013000000138301001302120093022000B8
:1002C000E31052FE930EF0FF130E40016314D30BA4
:1002D00013020000B700008093D170401302120097
:1002E00093022000E31852FEB70E00FF130E5001D8
:1002F0006392D10913020000B700008013000000D0
:1003000093D1E0401302120093022000E31652FE44
:10031000B70EFEFF130E6001639ED10513020000AD
:10032000B70000809380100013000000130000004D
:1003300093D1F0411302120093022000E31252FE07
:10034000930EF0FF130E70016396D103935040405B
:10035000930E0000130E8001639ED00193001002E3
:1003600013D0A040930E0000130E90016314D0012F
:10037000631CC0010F00F00F63000E00131E1E006F
:10038000136E1E00730000000F00F00F130E10001C
:1003900073000000731000C00000000000000000A7
:1003A000000000000000000000000000000000004D
:1003B000000000000000000000000000000000003D
:0403C0000000000039
:1010000000000000000000000000000000000000E0
:1010100000000000000000000000000000000000D0
:1010200000000000000000000000000000000000C0
:1010300000000000000000000000000000000000B0
:081040000000000000000000A8
:040000058000200057
:00000001FF
